:03000000020008F3
:0300610002000397
:0500030012006480FE04
:100064009000007401F07A017B0074F82B402AEAB6
:100074002400FCEB3400FDEA24FFFEEB34FFFFEE2A
:100084002400F582EF3400F583E0FE0E8C828D832C
:10009400EEF00ABA00D40B80D17A007B007C0074A5
:1000A400F82C4029EB2400F582EC3400F583E0FDC4
:1000B40074012BFEE43CE4FFF8EDB50606E8B50751
:1000C4000280030A8A800BBB00D50C80D2EA600749
:0F00D40075A0558AB0800675A0AA75B0AA80FEE7
:06003700E478FFF6D8FD9D
:100015007900E94400601B7A009000E7780075A03C
:1000250008E493F2A308B8000205A0D9F4DAF27542
:02003500A0FF2A
:10003D007800E84400600A790075A000E4F309D85F
:10004D00FC7800E84408600C7908900000E4F0A307
:04005D00D8FCD9FAF8
:0D0008007581071200E3E58260030200032A
:0400E3007582002200
:00000001FF
